:1000000000308A007E2C0000831A0A28A500030E07
:10001000A6000F288312A500030EA600A6140A0846
:10002000AD008A01A50E0408A7002008A800210839
:10003000A9002208AA002308AB002408AC00831200
:100040008C308400001E26280C1AC5288C308400B1
:10005000801E2C288C1ADC28270884002808A00081
:100060002908A1002A08A2002B08A3002C08A4003C
:10007000260E83008312250EA618831609000A1087
:100080008A100A11820720342034503469346334D2
:1000900053347534723466342034563431342E344B
:1000A00030342034203400340A108A100A118207B8
:1000B0005034683420342034553473345534663425
:1000C0002034203447345634443400340A108A1023
:1000D0000A11820741346C34613472346D346534F2
:1000E00020344C3449344134493453344F344E3441
:1000F000203400340A108A100A11820741346C340B
:10010000613472346D3465342034453441345534AF
:1001100000340A108A100A11820741346C346134A9
:1001200072346D3465342034623461347434203474
:10013000533455345234463400340A108A100A11AC
:10014000820741346C34613472346D346534203448
:10015000623461347434203446344F344E34443481
:1001600000340A108A100A11820720347034613476
:10017000733420346434273461346C346134723421
:100180006D346534733420340034E708031DCD2802
:1001900083160C1283120610D928670BD228E701A8
:1001A0009901D92855306607840000089900E60AAD
:1001B000E7030C128A112C2818080639003A031993
:1001C000E7285210181218161A08E8002E2952189B
:1001D000F3281A08023C031DF228F7010430F80046
:1001E000F90152142E296830770784001A0880001C
:1001F0006830770784000008F907F70A770B0329AE
:100200000530F8002E2978087702031C2E290130CA
:100210007702683E84000008033C0319112952103C
:100220002E290330F902790F1629182952102E2988
:1002300068087F398316B400831253087F39831608
:1002400034020319252983122929831254086902CB
:10025000031D2D296A08D100CB0A52108C128A1175
:100260002C28F701E7015210CA01CB016430CC0001
:100270000C30831699002430980090308312980037
:1002800083168C1683129B2C8316AC08031D4A29F7
:100290008312692983128316AE01AD01831283167E
:1002A000AE080319552983126529831283162D0878
:1002B000573C03185D2983126529831200008316B9
:1002C000AD0A0319AE0A83124F298316AC038312B9
:1002D0004429003403108316B20C83128316B20B28
:1002E000732983127629831200006E290034F030BE
:1002F00085058316310E8312A0000F30A00520085B
:10030000850486158611F0308505831631080F396E
:10031000831285048615861132308316B20083124B
:100320006A21003405120F308316AC008312442179
:10033000033085008615861105308316AC008312C4
:1003400044218615861164308316B20083126A2117
:100350008615861105308316AC00831244210230C5
:1003600085008615861128308316B20083126A2113
:1003700028308316B1008312772108308316B1002C
:10038000831277210C308316B10083127721063057
:100390008316B10083127721AC2CAD3084000008A5
:1003A0000319E1290130A100A001A00BD529A10B5F
:1003B000D4294A30A000A00BDB2900000000800BEC
:1003C000D2290034051201308316B100831277213F
:1003D00002308316AC0083124421003483162A08AD
:1003E00084002F088000840A8001AA0A8312003446
:1003F0000512803083162F07B000B10083127721D9
:1004000000348316AE012C08AF008312F821363079
:1004100083162E0784000008AD00AD08031D122AC4
:1004200083121D2A8312051683162D08B10083122C
:1004300077218316AE0A8312072A003406120613A8
:100440008316AC0DAC0DAC0DF830AC05C030AC046F
:10045000AD01831283162D08053C0318312A83123F
:100460004A2A831283162C088039803C03193A2AC1
:1004700083123D2A831286163E2A86120616031020
:100480008316AC0D00000000831206128316AD0A1D
:1004900083122A2A8316AD01831283162D08073C86
:1004A0000318542A83126B2A831203108316AE0D8D
:1004B0000000831206160030851A0130013C031D2E
:1004C000652A01308316AE078312000006128316D8
:1004D000AD0A83124D2A061783162E088312A10037
:1004E0000034831631088312A10183163002031CE5
:1004F0007B2A83127F2A30088312A000962AA0014B
:1005000008308316B20083128316B00D8312A00D3B
:1005100083163108831220020318A000A10D831650
:10052000B20B932A952A8312842A83120034A001E5
:10053000A101831630080310311CA12A8312A007E1
:1005400083168312A00CA10C8316B11CAA2A831255
:10055000A00783168312A00CA10C8316311DB32AA9
:100560008312A00783168312A00CA10C8316B11D61
:10057000BC2A8312A00783168312A00CA10C831639
:10058000311EC52A8312A00783168312A00CA10C6A
:100590008316B11ECE2A8312A00783168312A00CE5
:1005A000A10C8316311FD72A8312A007831683124A
:1005B000A00CA10C8316B11FE02A8312A00783169A
:1005C0008312A00CA10C003483162C08B0006430F8
:1005D000B1008312712221088316AF002D08AD0AE5
:1005E000840030302F0780002F08B0006430B10045
:1005F0008312972221088316AC022E0B002B022BAC
:1006000083120A2B831283162D08AD0A84002C3026
:100610008000831283162C08B0000A30B1008312C8
:10062000712221088316AF002D08AD0A84003030F6
:100630002F0780002F08B0000A30B10083129722E4
:1006400021088316AC022E08023C0319292B8312C1
:10065000312B831283162D08AD0A84002C308000C4
:10066000831283162D08AD0A840030302C078000D9
:100670002D0884008001831200348316AD0183129B
:100680000617061286120030851A0130003A031947
:100690004C2B83162D14831206160030851A013058
:1006A000003A0319562B8316AD14831206128616D0
:1006B0000030851A0130003A0319612B83162D157D
:1006C000831206160030851A0130003A03196B2B8D
:1006D0008316AD15831283162D08FF3A8312A100ED
:1006E0000034A030D300D4018316AD0155308312FD
:1006F000D5000230D6005308D7005408D80083161E
:10070000280D8312A000A00DFC30A0052008831640
:1007100029078312A000200ED000F030D005500829
:100720000138D9004F08DA004D08DB003E30DC000C
:100730004E08DD003E30DE00DF00E000E100023068
:100740008316AC00831283162C080C3C0318AA2BCA
:100750008312B62B8312553083162C0784000008B1
:10076000AD0783128316AC0A8312A32B83162D08C0
:100770008312E200E2090330E3005530E400772DF4
:1007800083162C08113C031CC72B8312C92B831220
:10079000E22BE7080319CD2BE22B06140130E6000B
:1007A00083162C088312E7005508990083160C164F
:1007B0008312CA0A4A08643C031DE22B4B08CC0092
:1007C000CA01CB017C2D3D2321088316A6002608F3
:1007D0002C052C020319EE2B8312002C8312831696
:1007E00027082C05003A0319F72B8312FF2B8312DD
:1007F00083162C08A70401308312A100072C052CB6
:1008000083162C08FF3AA70583120030A10000349C
:100810000516F030850583162D0E8312A0000F30CB
:10082000A0052008850486158611F03085058316FD
:100830002D080F39831285048615861132308316F0
:10084000B20083126A2100348316AD1F292C831253
:100850003C2CAD0803192E2C8312372C83128316DF
:100860002C081F3C031C362C83123C2C831283164D
:10087000AD011F30AC0083128316AD1B412C8312D7
:10088000582C2D08FF3C0318472C8312582C831238
:10089000031D522C83162C08E03C0318512C8312A4
:1008A000582C8312FF308316AD00E130AC00831268
:1008B0003E3083162C078312A10083162D08831265
:1008C000A3000318A30A2108003483162C083E3C19
:1008D00003196C2C8312702C83123030A1007D2CF4
:1008E00083162C083D3C0318772C83127B2C831233
:1008F0002D30A1007D2C2B30A100003484011F304D
:10090000830507309F00AE010130AF00B001B10197
:10091000B2018316AA018312A0308316850002302B
:100920008600831285018030860007309F003030BA
:10093000900064003129C0308B003E30CD00CE00E5
:10094000CF00D001D1018316A901A801A701A601FA
:1009500083125211D210922964308316AD00831293
:10096000CD21E22164308316AD008312CD213630D3
:100970008316AA00AC01831283162C0883123F2031
:100980008316AC0AAF008312EE21103083162C02BE
:100990000319CC2C8312BC2C8312861304308316CB
:1009A000AC008312FA308316AD008312CD2183167A
:1009B000AC0BDB2CDD2C8312D22CAC018312012278
:1009C00004308316AC008312FA308316AD00831214
:1009D000CD218316AC0BED2CEF2C8312E42C83126B
:1009E000E2217F30FD00FE00FF008316AC01831280
:1009F0001E222108FA0004308316AC0083121E2246
:100A00002108FB0001308316AC0083121E2221084E
:100A1000FC007A088316AC003730AD00AE018312BB
:100A2000E4225830B6008316AC01831201227B0801
:100A30008316AC003730AD00AE018312E42259308A
:100A4000B60005308316AC00831201227C088316A1
:100A5000AC003730AD00AE018312E4225A30B6004C
:100A60000A308316AC00831201223D232108043989
:100A7000003A031DF52CE22136308316AA00AC01A2
:100A8000831283162C08831254208316AC0AAF00FD
:100A90008312EE21063083162C020319512D831286
:100AA000412D0330AD00831220308316AF00831236
:100AB000EE218316AD0B5D2D5F2D8312542D063074
:100AC000AE00831283162E08831254208316AE0ABA
:100AD000AF008312EE210D3083162E020319722D02
:100AE0008312622DAC01831201226400712B10303D
:100AF0008316AC008312C02B07308316AC00831220
:100B00001E222108C80003308316AC0083121E2267
:100B10002108C9008316AC0183121E222108FA00A5
:100B200004308316AC0083121E222108FB00013022
:100B30008316AC0083121E222108FC0002308316AB
:100B4000AC008312E323210BDE2D8316A90A2908AA
:100B5000033C031CAD2D8312B12D83128316A90112
:100B6000831240308316AF008312F82183162908C0
:100B70000139003A031DBE2D8312C52D8312313079
:100B80008316AD0083120824CA2D20308316AD00D1
:100B900083120824831629080239003A031DD22D36
:100BA0008312D92D831232308316AD0083120824AC
:100BB000DE2D20308316AD00831208240830831602
:100BC000AC008312E323210BE62DD2147F087C02B4
:100BD0000318FB2D7C087F02FC00FC0CFC0C3F3052
:100BE000FC057C083E3CCF004F081E3C031CFA2D40
:100BF0001F30CF000A2E7F08FC02FC0CFC0C3F309B
:100C0000FC053E307C07CF004F085E3C03180A2EDF
:100C10005E30CF008316AD0183127A088316AC00D4
:100C20008312A3017D0883162C02A0002D08A100C9
:100C300083122308031C230F1E2E212E8316A102CC
:100C400083128316AD0183127B088316AC008312D6
:100C5000A3017E0883162C02A2002D08A300831294
:100C60002308031C230F352E382E8316A30283126C
:100C7000831620082207A4002308A5000318A50A4C
:100C80002108A5072508AD002408AC008312242400
:100C90002108CE00831620082202A4002308A50004
:100CA0002108031C210FA5022508AD002408AC0073
:100CB000831224242108CD004E088316AC00363060
:100CC000AD00AE018312E42210308316AC00831213
:100CD00001224F088316AC003630AD00AE018312FE
:100CE000E42217308316AC00831201224D088316CC
:100CF000AC003630AD00AE018312E4221D30831605
:100D0000AC008312012248088316AC003630AD00D7
:100D10000230AE008312E42243308316AC0083120B
:100D2000012249088316AC003630AD000230AE0017
:100D30008312E42248308316AC00831201224D3026
:100D40008316AF008312F8214E088316AC0083127D
:100D5000652421088316AC00AD00831208244F08D7
:100D60008316AC008312652421088316AC00AD0005
:100D7000831208244D088316AC00831265242108D1
:100D80008316AC00AD00831208244C08313C031CD0
:100D9000E42E36308316AA00AC01831283162C0889
:100DA000831266208316AC0AAF008312EE210F3047
:100DB00083162C020319DE2E8312CE2E5030AC0087
:100DC0008312012252156B2F51080F39003A031973
:100DD000122F36308316AA00AC01831283162C081A
:100DE00083127A208316AC0AAF008312EE210A30F8
:100DF00083162C020319FE2E8312EE2E0530AD0051
:100E0000831220308316AF008312EE218316AD0BC0
:100E10000A2F0C2F8312012F5030AC0083120122B5
:100E200052156B2F4808723C031C312F3630831645
:100E3000AA00AC01831283162C0883128920831622
:100E4000AC0AAF008312EE210F3083162C02031977
:100E50002B2F83121B2F5030AC008312012252150E
:100E60006B2F4908E53C031C502F36308316AA002F
:100E7000AC01831283162C0883129D208316AC0AC2
:100E8000AF008312EE210F3083162C0203194A2F74
:100E900083123A2F5030AC008312012252156B2F6F
:100EA00036308316AA00AC01831283162C088312F5
:100EB000B1208316AC0AAF008312EE210F308316E7
:100EC0002C020319652F8312552F5030AC0083126A
:100ED00001225211D210003052190130013C031D81
:100EE000792F0030D2180130003A031D792F861770
:100EF0007A2F86131E308316AD008312CD21752DF7
:020F000063008C
:02400E00413F30
:00000001FF
